:10000000B401742A9221B6000408B80008009221B5
:10001000B7000408B90008000408A200831686117E
:1000200083120930A30003101C20A20CA30B142878
:1000300003141C2003146F2A0318212800008615BE
:100040002328861123280030A100C330DD290408AD
:10005000A7000610861086108316061086108610DC
:100060000F30860583122708B41854283A30A100AF
:100070009830DD213330A60068201330A10088308D
:10008000DD2168206430DC2168206430DC212230EE
:10009000A6006820283053200C305320063053200F
:1000A000B414270854283414A600341C622886107F
:1000B000033C031C672867200730A100D030DD21F6
:1000C000031408003414FE3C03196F2A8614341CF0
:1000D000341006140F3086052608F0398604061001
:1000E000A60E341868283230DC210314080092214F
:1000F000B6008E212008210403196F2A642284137C
:1001000036088006640084288528A00A0319A10FF8
:10011000822880066F2A6400A12003188B28EE2015
:10012000A8010830A300EF20A1200318A80AAB1EE5
:10013000A801A20CA30B9328AB1AA213EF2022084C
:1001400008003808840036088417800484130005EA
:100150002B1B3606FF3E0800290803196F2A6A2266
:10016000A903AC28A401A501B5126A22D33E031944
:10017000B5162D3EC63E0318C1280A3E031CB528FD
:10018000C828F33E0318B528063E031CB5280A3ECE
:10019000A2000430A3000310A40DA50DA30BCB28CF
:1001A0002208A404A9030319E5286A22C63E0318FD
:1001B000DD280A3E031CE528C828F33E0318E5287D
:1001C000063E031CE5280A3EC828B51EEC28A409F3
:1001D000A509A40A0319A50A24086F2A35172B08B4
:1001E0001F39FF3EA1002A08F53E0318A10A351F5A
:1001F000DD293513A00002300F22DD29B5132908AF
:100200000319B5170430A800250E0B2125080B2172
:10021000240E0B2124080F39F63E0318073E0A3E30
:100220002E29B51329080319B5170530A800273062
:10023000A300103027210330A300E8302721A301B9
:1002400064302721A3010A30272124082E29A20087
:100250002508A1002408A00032222008A000A8033D
:100260000319B513290803193829280203180800AF
:100270002008031DB513B51B0800303E6A2A08305C
:10028000A600A70039088400370835198004FF3A12
:10029000351D80058F213808840036088B21A00188
:1002A000A101B5187F213808840000083605FF3EFB
:1002B000A00DA10DB51C7F21A60B512927083518CB
:1002C000F12920086F2A0830A6003518F1213908D5
:1002D0008400370835198621351D882138088400A7
:1002E00036098F2138088400A10CA00C00083604C0
:1002F000031C360680007F21A60B72296F2A39085D
:1003000084003708800600008006080080048E29DB
:10031000FF3A80058F29841780046F2AFF3A8417DB
:1003200080056F2AA8000630A81907308400013024
:100330008A0028080739820701340234043408345B
:100340001034203440348034A000A00DA00DA00D46
:100350003830A005813020049F000030A1003230E9
:10036000DD211F151F19B2291E08A10083161E08C2
:100370006F2A03178D0083168C130C1483120C083C
:100380006F2A03178C0083168C130C1555308D00C3
:10039000AA308D008C148C18CB290C116F2AA30164
:1003A000A200FF30A207031CA307031C6F2A03301F
:1003B000A100DF30DD21D129A101E83EA000A10983
:1003C000FC30031CE629A0070318E329A0076400FA
:1003D000A10FE3292018EC29A01CF0290000F02926
:1003E0000800A400A201A301F929A10CA00CA20DF0
:1003F000A30DFF3E0318F529240807222208A004B4
:100400002308A104200808000310A00DA10DFF3E41
:100410000318042A20086F2A0310A10CA00CFF3E29
:1004200003180C2A20086F2AA2000330222AA200F7
:100430000130222AA2000630222AA2000430222AF9
:10044000A2000530A80023082102031D292A220842
:100450002002043003180130031902302805031D5F
:10046000FF306F2A1030A600A501A401210DA40DB4
:10047000A50D2208A4022308031C230FA5020318BC
:10048000482A2208A40723080318230FA5070310EE
:10049000A00DA10DA60B362A20086F2A1030A80047
:1004A000A101A001A70CA60C031C5C2A2208A0072E
:1004B00023080318230FA107A10CA00CA50CA40C62
:1004C000A80B522A24086F2AA009A109A00A03191F
:1004D000A10A0800840031088A00300882008313D2
:1004E00003138312640008000330A300E8308A017C
:1004F000D0218316043086003F308500FC30870011
:100500008312831684309F00831281309F006430F1
:10051000FE00FD016430F400F3011F30C20004301E
:10052000C3002030C0000330C1000130BC00BD0159
:100530000130EE0064008A110A12071EA62A640028
:100540008A110A12071A632F8A019A2AFE308A0139
:10055000282001308A01282043308A012820613078
:100560008A0128206C308A01282069308A012820DD
:1005700062308A01282072308A01282061308A0185
:10058000282063308A01282069308A0128206F30B2
:100590008A0128206E308A01282043308A010D20EC
:1005A00061308A010D206C308A010D2069308A018A
:1005B0000D2062308A010D2072308A010D206130D9
:1005C0008A010D2063308A010D2069308A010D20D7
:1005D0006F308A010D206E308A010D2020308A0193
:1005E0000D202D308A010D2020308A010D2065302C
:1005F0008A010D206E308A010D2074308A010D2091
:1006000072308A010D2061308A010D2072308A011A
:100610000D2020308A010D2076308A010D206130B6
:100620008A010D206C308A010D206F308A010D2067
:1006300072308A010D2065308A010D2073308A01E5
:100640000D200A308A010D200D308A010D20433023
:100650008A010D206F308A010D206D308A010D2036
:1006600070308A010D2065308A010D206E308A01BC
:100670000D2073308A010D2061308A010D20633016
:100680008A010D2069308A010D206F308A010D200A
:100690006E308A010D2020308A010D2054308A01ED
:1006A0000D2065308A010D206D308A010D207030DB
:1006B0008A010D202B308A010D203A308A010D204D
:1006C0000A308A010D200D308A010D200530B80056
:1006D0002030B600BC30AA004030AB000130A90089
:1006E0008B30B000B1018A01B220F8000130A900BE
:1006F0007808A400A5010C30B000B1018A01FE20E9
:100700000A308A010D200D308A010D20FE308A0149
:100710002820C0308A01282054308A0128206530E2
:100720008A0128206D308A01282070308A01282013
:1007300020308A0128202B308A0128200130A9008E
:100740007808A400A5012730B000B1018A01FE207D
:10075000031701308D00031378088A01C12103308B
:10076000A300E8308A01D021FE308A012820013020
:100770008A01282043308A01282061308A012820FC
:100780006C308A01282069308A01282062308A0171
:10079000282072308A01282061308A0128206330A5
:1007A0008A01282069308A0128206F308A01282098
:1007B0006E308A01282043308A010D206F308A0173
:1007C0000D206D308A010D2070308A010D206530BA
:1007D0008A010D206E308A010D2073308A010D20B0
:1007E00061308A010D2063308A010D2069308A0151
:1007F0000D206F308A010D206E308A010D202030CF
:100800008A010D2054308A010D2065308A010D20A7
:100810006D308A010D2070308A010D202D308A0143
:100820000D203A308A010D200A308A010D200D304A
:100830008A010D200530B8002030B600BC30AA0077
:100840004030AB000130A9008B30B000B1018A010B
:10085000B220F8000130A9007808A400A5010C30EE
:10086000B000B1018A01FE200A308A010D200D304E
:100870008A010D20FE308A012820C0308A012820FC
:1008800054308A01282065308A0128206D308A0181
:10089000282070308A01282020308A0128202D301D
:1008A0008A0128200130A9007808A400A50127307A
:1008B000B000B1018A01FE20031702308D0003133E
:1008C00078088A01C1210330A300E8308A01D021D1
:1008D000FE308A01282001308A01282043308A0115
:1008E000282061308A0128206C308A012820693054
:1008F0008A01282062308A01282072308A0128204B
:1009000061308A01282063308A01282069308A01F9
:1009100028206F308A0128206E308A012820433039
:100920008A010D206F308A010D206D308A010D2063
:1009300070308A010D2065308A010D206E308A01E9
:100940000D2073308A010D2061308A010D20633043
:100950008A010D2069308A010D206F308A010D2037
:100960006E308A010D2020308A010D2048308A0126
:100970000D2075308A010D206D308A010D202B303D
:100980008A010D203A308A010D200A308A010D209B
:100990000D308A010D200530B8002030B600BC3083
:1009A000AA004030AB000130A9008B30B000B1018B
:1009B0008A01B220F8000130A9007808A400A5013E
:1009C0000C30B000B1018A01FE200A308A010D20EE
:1009D0000D308A010D20FE308A012820C0308A01A6
:1009E000282048308A01282075308A0128206D305F
:1009F0008A01282020308A0128202B308A012820D3
:100A00000130A9007808A400A5012730B000B10189
:100A10008A01FE20031703308D00031378088A0132
:100A2000C1210330A300E8308A01D021FE308A01C1
:100A3000282001308A01282043308A012820613093
:100A40008A0128206C308A01282069308A012820F8
:100A500062308A01282072308A01282061308A01A0
:100A6000282063308A01282069308A0128206F30CD
:100A70008A0128206E308A01282043308A010D2007
:100A80006F308A010D206D308A010D2070308A018F
:100A90000D2065308A010D206E308A010D207330E3
:100AA0008A010D2061308A010D2063308A010D20FA
:100AB00069308A010D206F308A010D206E308A0165
:100AC0000D2020308A010D2048308A010D2075301C
:100AD0008A010D206D308A010D202D308A010D20F4
:100AE0003A308A010D200A308A010D200D308A012A
:100AF0000D200530B8002030B600BC30AA004030D0
:100B0000AB000130A9008B30B000B1018A01B220E6
:100B1000F8000130A9007808A400A5010C30B0004D
:100B2000B1018A01FE200A308A010D200D308A01B0
:100B30000D20FE308A012820C0308A01282048304C
:100B40008A01282075308A0128206D308A012820EA
:100B500020308A0128202D308A0128200130A90068
:100B60007808A400A5012730B000B1018A01FE2059
:100B7000031704308D00031378088A01C121033064
:100B8000A300E8308A01D021FE308A0128200130FC
:100B90008A01282043308A01282061308A012820D8
:100BA0006C308A01282069308A01282062308A014D
:100BB000282072308A01282061308A012820633081
:100BC0008A01282069308A0128206F308A01282074
:100BD0006E308A01282043308A010D206F308A014F
:100BE0000D206D308A010D2070308A010D20653096
:100BF0008A010D206E308A010D2073308A010D208C
:100C000061308A010D2063308A010D2069308A012C
:100C10000D206F308A010D206E308A010D202030AA
:100C20008A010D2050308A010D2072308A010D207A
:100C300065308A010D2073308A010D2073308A01DE
:100C40000D202B308A010D203A308A010D200A3008
:100C50008A010D200D308A010D200530B8002030AA
:100C6000B600BC30AA004030AB000130A9008B3088
:100C7000B000B1018A01B220F8000130A900780863
:100C8000A400A5010C30B000B1018A01FE200A3099
:100C90008A010D200D308A010D20FE308A012820A6
:100CA000C0308A01282050308A01282072308A0101
:100CB000282065308A01282073308A01282073306B
:100CC0008A01282020308A0128202B308A01282000
:100CD0000130A9007808A400A5012730B000B101B7
:100CE0008A01FE20031705308D00031378088A015E
:100CF000C1210330A300E8308A01D021FE308A01EF
:100D0000282001308A01282043308A0128206130C0
:100D10008A0128206C308A01282069308A01282025
:100D200062308A01282072308A01282061308A01CD
:100D3000282063308A01282069308A0128206F30FA
:100D40008A0128206E308A01282043308A010D2034
:100D50006F308A010D206D308A010D2070308A01BC
:100D60000D2065308A010D206E308A010D20733010
:100D70008A010D2061308A010D2063308A010D2027
:100D800069308A010D206F308A010D206E308A0192
:100D90000D2020308A010D2050308A010D20723044
:100DA0008A010D2065308A010D2073308A010D20E3
:100DB00073308A010D202D308A010D203A308A01CE
:100DC0000D200A308A010D200D308A010D200530DA
:100DD000B8002030B600BC30AA004030AB00013073
:100DE000A9008B30B000B1018A01B220F8000130B7
:100DF000A9007808A400A5010C30B000B1018A0157
:100E0000FE200A308A010D200D308A010D20FE30AF
:100E10008A012820C0308A01282050308A012820E9
:100E200072308A01282065308A01282073308A01B7
:100E3000282073308A01282020308A0128202D3074
:100E40008A0128200130A9007808A400A5012730D4
:100E5000B000B1018A01FE20031706308D00031394
:100E600078088A01C1210330A300E8308A01D0212B
:100E7000FE308A01282001308A01282050308A0162
:100E8000282075308A0128206C308A012820733090
:100E90008A01282061308A01282072308A012820A6
:100EA00020308A01282052308A01282065308A01AA
:100EB000282073308A01282065308A012820743068
:100EC0008A0128200800FE308A01282001308A018A
:100ED000282057308A01282045308A0128204130B7
:100EE0008A01282054308A01282048308A0128208D
:100EF00045308A01282052308A01282020308A017A
:100F0000282020308A01282053308A01282054309C
:100F10008A01282041308A01282054308A01282063
:100F200049308A0128204F308A0128204E308A011A
:100F30002820FE308A012820C0308A012820453030
:100F40008A01282041308A01282033308A01282054
:100F500043308A0128204E308A0128204F308A01F0
:100F6000282020308A01282020308A0128202030A3
:100F70008A01282050308A01282049308A012820FF
:100F800043308A0128205F308A01282057308A01A7
:100F9000282058308A01282043308A0128200B302D
:100FA000A300B8308A01D0218716831687120F302C
:100FB00083128A0102200E308A010720B5010C300D
:100FC000A000A1018A0163210230A000A1018A01D1
:100FD0006321871283168712831200308A01A421AD
:100FE000E60001308A01A421BA002108BB000330C9
:100FF0008A01A421E7000530B8000430B600BC30F7
:10100000AA004030AB008A018B202A3C8A150A12C4
:10101000031D03280230A9008B30B000B1018A0102
:10102000B220F1000130A9008B30B000B1018A017B
:10103000AC200230A9008B30B000B1018A01B2208F
:10104000F5000130A9008B30B000B1018A01AC205D
:101050000230A9008B30B000B1018A01B220F90042
:101060000130A9008B30B000B1018A01AC20023000
:10107000A9008B30B000B1018A01B220EF0001302D
:10108000A9008B30B000B1018A01AC200230A90068
:101090008B30B000B1018A01B220F6000130A90006
:1010A0008B30B000B1018A01AC200230A9008B3036
:1010B000B000B1018A01B220FF0001308A01B921DC
:1010C000ED0002308A01B921EC0003308A01B92118
:1010D000E90004308A01B921E80005308A01B9210C
:1010E000EB0006308A01B921EA008A150A12202293
:1010F0008A150A125E228A150A1276228A150A12A7
:10110000F4228A150A1212233E08A0003F08A1000B
:101110004508A30044088A011A228A150A12031DF1
:1011200093287E30F0003E08A0003F08A10045084B
:10113000A30044088A0120228A150A12031DA2284E
:101140003D30F0003E08A0003F08A1004508A30084
:1011500044088A0114228A150A12031DB1287F301F
:10116000F000FE308A01282001308A01282020303A
:101170008A0128202B308A0128200230A9007A0811
:10118000A400A5012730B000B1018A0111212E3041
:101190008A0128200130A9007C08A400A50127307D
:1011A000B000B1018A011121DF308A0128204330CB
:1011B0008A01282020308A01282020308A01282016
:1011C0000230A9007208A400A5012730B000B101C7
:1011D0008A01112125308A01282052308A012820D5
:1011E00048308A01282020308A012820FE308A01D8
:1011F0002820C0308A01282020308A012820203071
:101200008A01282020308A0128200430A9003E08C5
:10121000A4003F08A5002730B000B1018A011121C8
:1012200020308A01282068308A01282050308A0125
:10123000282061308A01282020308A012820700867
:101240008A01282020308A01282020308A01282085
:1012500020308A0128200A308A01CF2164008A15B3
:101260000A12871D712B64008A150A12071EF22BC1
:101270008A150A1222238A150A1237238A150A129E
:101280004C23BC0A0319BD0A3C08A0003D08A1007C
:101290000130A3002B308A011D228A110A12031D7E
:1012A000ED2F2E308A010D202E308A010D202E3098
:1012B0008A010D202C308A010D202E308A010D204C
:1012C0002E308A010D202E308A010D202C308A010B
:1012D0000D202E308A010D202E308A010D202E3057
:1012E0008A010D202C308A010D200330A9004A0804
:1012F000A4004B08A5000C30B000B1018A011121F7
:101300002C308A010D200430A9003E08A4003F08BB
:10131000A5000C30B000B1018A0111212C308A01E6
:101320000D200230A9007208A400A5010C30B00005
:10133000B1018A0111212C308A010D200230A9004F
:101340006F08A400A5010C30B000B1018A01FE2095
:101350002C308A010D200230A9007108A400A501DB
:101360000C30B000B1018A01FE202C308A010D2022
:101370000230A9007508A400A5010C30B000B1012D
:101380008A01FE202A308A010D202E308A010D208C
:101390002E308A010D202E308A010D202C308A013A
:1013A0000D202E308A010D202E308A010D202E3086
:1013B0008A010D202C308A010D202E308A010D204B
:1013C0002E308A010D202E308A010D202A308A010C
:1013D0000D202A308A010D200230A9007A08A400CD
:1013E000A5010C30B000B1018A0111212E308A0113
:1013F0000D20A9017C08A400A5010C30B000B101AA
:101400008A0111210A308A010D200D308A010D2038
:101410000130BC00BD01EE0A64000B306E028A117F
:101420000A12031CED2F3E08C4003F08C50001301E
:10143000EE000330A300E8308A01D0218A01ED2FAD
:101440008716831687120F3083128A0102200E300E
:101450008A010720B501EE30A000A1018A016321B5
:1014600087128316871283128716831687120F300E
:1014700083128A0102200E308A010720B501AA30AA
:10148000A000A1018A0163210F308A0102200E30E1
:101490008A0107200130B5008A013F21CA002108D6
:1014A000CB0087128316871283126D08CA070318B0
:1014B000CB0A6C08CA02031CCB0308004B0C4A0C75
:1014C000FA004A08A0004B08A1000230A200A301C4
:1014D0008A0132222408FB007B08A600A701053000
:1014E000A200A3018A014E22FC0008003A08A600CF
:1014F0003B08A7003230A200A3018A014E22B200AD
:101500002508B3003208A0003308A100FF30A20074
:101510000330A3008A013222C6002108C7003A081E
:10152000A6003B08A7003230A200A3018A014E2288
:10153000B2002508B3003208A0003308A100FF3034
:10154000A2000330A3008A0132222408C800250823
:10155000C9004608A6004708A700E830A2000330EB
:10156000A3008A014E22B2002508B3004808B20742
:1015700049080318013EB3073208A0003308A10050
:10158000F430A2000130A3008A013222B200210807
:10159000B3001030B2020030031C013EB302320827
:1015A000A6003308A7006430A200A3018A014E22DE
:1015B000B2002508B3003208A0003308A1003E3075
:1015C000A200A3018A013222F2006908F20768082A
:1015D000F2026400633072028A150A120318F12ABB
:1015E00008006330F200080007108316071083120A
:1015F00087108316871083126430A000A101093080
:101600008A0177200A308A01022009308A010720E6
:101610000230B5008A013F21F70007148316071036
:101620008312080020307707BE0003300318013E04
:10163000BF006B08BE070318BF0A6A08BE02031C7E
:10164000BF03080064007A087D028A150A12031C91
:10165000312B64007E087A028A150A12031C342B8F
:1016600008007A08FD0008007A08FE0008006400FF
:10167000720873028A150A12031C462B6400740850
:1016800072028A150A12031C492B08007208F30023
:1016900008007208F40008003E08A0003F08A100FE
:1016A0004108A30040088A0117228A150A12031D67
:1016B000672B3E08A0003F08A1004308A300420892
:1016C0008A011D228A150A12031D6C2B08003E0890
:1016D000C0003F08C10008003E08C2003F08C30028
:1016E0000800FE308A01282001308A012820DF30DE
:1016F0008A01282043308A01282020308A012820AE
:1017000020308A01282020308A0128204D308A018B
:10171000282020308A0128202B308A0128200230FE
:10172000A9007D08A400A5012730B000B1018A01FD
:10173000112120308A0128206D308A012820203094
:101740008A0128202B308A0128200230A9007E0837
:10175000A400A5012730B000B1018A011121FE309B
:101760008A012820C0308A01282025308A012820BB
:1017700052308A01282048308A01282020308A01EE
:10178000282020308A0128204D308A01282020304E
:101790008A01282020308A0128200230A9007308FD
:1017A000A400A5012730B000B1018A011121203029
:1017B0008A0128206D308A01282020308A012820C3
:1017C00020308A0128200230A9007408A400A50155
:1017D0002730B000B1018A01112164308A01CF2184
:1017E0008A01ED2FFE308A01282001308A0128204D
:1017F00068308A01282050308A01282061308A010F
:10180000282020308A01282020308A0128204D30CD
:101810008A0128200430A9004008A4004108A5003E
:101820002730B000B1018A01112120308A0128201F
:101830006D308A0128200430A9004208A400430822
:10184000A5002730B000B1018A011121FE308A01C4
:101850002820C0308A01282020308A012820023028
:10186000A9007108A400A5012730B000B1018A01C8
:10187000FE203A308A0128200230A9007508A40011
:10188000A5012730B000B1018A01FE2020308A0175
:1018900028200230A9006F08A400A5012730B0005D
:1018A000B1018A01FE202F308A0128200230A900D0
:1018B0007608A400A5012730B000B1018A01FE20FE
:1018C0002F308A0128200230A9007F08A400A5013A
:1018D0002730B000B1018A01FE2064308A01CF2197
:0418E0008A01ED2F5D
:02400E00753DFE
:00000001FF
